:103400000C94DE1A002700BD07E109B908E10AB9EA
:1034100006E800BD08955D9BFECF4CB908955F9B03
:10342000FECF4CB10895C895002021F0402DF3DF68
:103430003196F9CF0895C895002021F0402DEBDF9B
:103440003296F9CF0895C895002021F0501519F053
:103450003296F9CF08940895C895002041F0501590
:1034600011F03296F9CF3196C895C02C8C2C089566
:10347000C895002039F0501511F03296F9CF3196E9
:10348000C895D02C089518E22DE32A95F1F71A95E6
:10349000D9F70A95C1F708951AD03D2F18D03C2FBF
:1034A00016D00895312D13D0322D11D0332D0FD0D9
:1034B000342F0DD00895312D0AD0322D08D0332D60
:1034C00006D004D0432F03D0A6DF0895332708E0A9
:1034D00070E0331F10F4C59A01C0C598770FB699F4
:1034E0007160C79A1AE01A95F1F7C79815E01A9516
:1034F000F1F70A9571F7372F0895552322F030E23E
:10350000E6DF3D2F03C03D2F41D03160E0DF3C2F8F
:10351000DEDFDCDF432F7FDF55234AF038E2D7DFE1
:103520003D2FD5DF3C2FD3DFD1DF432F74DF219632
:103530000895552322F030EACADF3D2F05C05738E1
:1035400059F03D2F23D03560C2DF3C2FC0DFBEDFF6
:10355000432F61DF219608950F910F91B4C2552337
:1035600022F030ECB4DF3D2F05C0573861F03D2F1D
:103570000DD03660ACDF3C2FAADF342FA8DF0AE085
:1035800082DF219608950F910F919DC2330F330F63
:10359000330F18F4573809F434600895C39A08ECCF
:1035A00072DF08EC70DF34E1C39805E06CDFC39A8A
:1035B00002E369DF3A95C1F7C39A08950FE50DBF9D
:1035C00004E00EBF00270BBF1DDFBB9A0FEF02BB4D
:1035D00008BBB898C098E2DF1BEA17BBC0981FDF92
:1035E0004B31E9F3443559F41ADF542FE2EFFAE393
:1035F00033DF0FEFD02EE2EDFAE33ADF67C2433557
:1036000021F4E4E3FBE30FDFEACF463521F4ECE2FB
:10361000FBE309DFE4CF463721F4E0E3FBE303DF1C
:10362000DECF443749F4E2EDFAE305DFE2EFFAE3F7
:1036300002DF40E0F0DED3CF403719F443E5EBDEA4
:10364000CECF413619F449E5E6DEC9CF493631F42B
:10365000ECE3FBE3E8DE4AE0DEDE38C2423639F472
:1036600049E5D9DE40E0D7DE40E4D5DEB8CF4837C3
:1036700019F4D5DEC3982AC2493719F4D0DEC39AAB
:1036800025C2E2EDFAE3DFDE28F4E2EFFAE3DBDE67
:1036900008F419C2403509F03BC0C39812E011BBD1
:1036A0001AEA17BBC098C798552312F0C19A01C0F7
:1036B000C19802E3E8DE552312F0C19801C0C19A17
:1036C00002E3E1DE3CEA03DF33E501DF5032B8F02C
:1036D0005523AAF020E2FADE333599F030E0F7DE28
:1036E000C79A1AE01A95F1F7C79815E01A95F1F7FD
:1036F0003CEAEDDE33E5EBDE2A9569F702C030E007
:10370000E6DE552312F030E0E2DE04E0BCDEDEC18E
:103710004336B9F484DE30E4832F55231AF0D7DE24
:103720003D2F03C03D2F32DF3260D1DE3C2FCFDE94
:10373000342FCDDE942F4C2E5D2E55230AF4219686
:103740006BC1433491F46BDE552372F038E4832F60
:10375000BEDE3D2FBCDE3C2FBADE342FB8DE942F08
:103760004C2E5D2E219658C1AEC1423409F073C073
:1037700056DE442311F041E0A6C151DE413410F081
:1037800042E0A1C1642E742E4ADEB42EBB27A0E60F
:1037900046DE4D936A94E1F7BB27A0E621E0A22E16
:1037A0004B2D463449F0453411F043E08CC14D9126
:1037B000D6DE7A94E1F78AC1E2EFFAE344DE08F458
:1037C00023C030E469DE3D9182DE38E4832F64DE7D
:1037D0003D91932F4C2E5D2E7ADE21967A9431F016
:1037E0007A9421F0AA2069F38A9459F7AA2009F45F
:1037F0006DC18A943CE46BDE352D69DE342D67DEC5
:1038000030E065DE8C2C31C15523DAF09D919F3F6D
:1038100041F030E4832F40DE392F59DE4C2E5D2EEF
:1038200000D17A949D919F3F41F038E4832F34DE9C
:10383000392F4DDE4C2E5D2EF4D021967A9421F74F
:1038400045C13D2FA3DE326042DE3C2F40DE3D917C
:10385000932F3DDEEFCF4235E1F4552322F038E2DD
:1038600036DE3D2F03C03D2F91DE316030DE3C2F30
:103870002EDE2CDE432FCFDD55234AF030E227DE4B
:103880003D2F25DE3C2F23DE21DE432FC4DD219694
:10389000A6CE4736B9F4C3DDB42FC1DDA42FBFDDFA
:1038A000463439F0453409F00EC143DE1197E9F78B
:1038B00096CE23DE55231AF01297D9F790CE1197A2
:1038C000C1F78DCE413429F4AADDD42FA8DDC42F51
:1038D000FDC0443419F4A3DD42DEF8C0443611F4CF
:1038E00028DE7DCE4C3471F4552312F0C19A01C00C
:1038F000C1981BEA17BBC098C39A0EEF08BBB89AD1
:10390000C098E4C0453409F4EFCF453669F43CEA89
:10391000DEDD552312F030E8DADD34E0D8DD30E0CA
:10392000D6DD08E2B0DDD2C04C36F9F478DD3CEAF1
:10393000CEDD55238AF05E3539F0342F3670306E87
:10394000C6DD30E0C4DD0CC030EEC1DD30E0BFDDEF
:10395000342F3C6FBCDD06C0342F307E3760B7DDBE
:1039600030E0B5DD0AE08FDDB1C04337A1F4552367
:103970003AF062E006D061E004D060E002D02FCEE1
:10398000A2C030E3A4DD30E0A2DD362FA0DD9EDD55
:10399000432F41DD08954D3649F43CE498DD352D43
:1039A00096DD342D94DD30E092DD5FC04A3391F432
:1039B00036DD142E34DD242E32DD342E312D87DD1C
:1039C000322D85DD332D83DD81DD432F24DD02E3C0
:1039D0005ADD7CC04E32A1F422DD142E20DD242ECF
:1039E0001EDD342E1CDD312D72DD322D70DD332DC8
:1039F0006EDD342F6CDD472F0EDD02E344DD66C043
:103A0000423749F438E563DD332761DD60DD5EDD93
:103A1000432F01DD5BC057C0E2EFFAE314DD18F07D
:103A200055C021E0922EDD20D1F09D15C1F08F70A0
:103A300080622227552322F0382F49DD352D03C01F
:103A4000352DA4DD316043DD342D41DD3FDD5523CF
:103A500012F430789078391721F02A9559F70AE056
:103A600012DD992099F199240895513499F0533237
:103A7000D1F09F3F79F08F7080622227382F27DDA9
:103A8000352D25DD342D23DD21DD391729F02A954B
:103A900009F0F4CF02E3F7DCAA2019F0772009F04F
:103AA00090CEAA2413C080EF2227522E382F0FDD8C
:103AB000352D0DDD342D0BDD09DD317069F32A95CF
:103AC00049F3F4CFA8DC4FE3A6DC89CD4DE0A3DCBD
:103AD00086CD1300207F287F30FF34FF387F48FFDA
:103AE0004CFF51FF55FF56FF68FF6CFF86FF87FFB5
:103AF000000023103A203B204140434044404540D1
:103B000046405E10604061406240634064406640F1
:103B100069206A2072407340744075407620772097
:103B20007840794065206720424000003130000035
:103B30003130000041565220495350005665722ED4
:103B4000312E30204156522044554F2049434500E4
:103B50004D43552050726F53686F7000FFFFFFFF99
:00000001FF
